:020000040000FA
:020000003528A1
:080008000428051D0D28851ECA
:100010001328051E19281F2005280510851005190D
:1000200005281F200F2805148510851A05281F2074
:10003000152805108514051A05281F201B280230D5
:10004000A5007F30A400A50B26282A282B20A40B6E
:100050002628212808000130A000C830013C003CBF
:10006000031D2E28A00B2D280800831285018B016B
:100070000730990000309F00831600309F008C01EC
:10008000960195010F3081003C3085008312850177
:100090000330A300FF3085001F20003085001F20A3
:0A00A000A30B4A2800308500052854
:02400E00843FED
:024200000800B4
:00000001FF
